:080000000C9448000C94000070
:100008000C9400000C9400000C9400000C94000068
:100018000C9400000C9400000C9400000C94000058
:100028000C9400000C9400000C9400000C94000048
:100038000C9400000C9400000C9400000C94000038
:100048000C9400000C9400000C94000020202569FA
:10005800205320746F206F6E2020002020616D696E
:100068006E20666172686F64692020001027E803BB
:1000780064000A0001000010000110000100600186
:10008800020080C086000000F894EE27ECBBF1E087
:10009800FBBFEBBFE5BFF8E1F1BDF0E1F1BD8DE0DD
:1000A800A2E0BB27ED938A95E9F780E094E0A0E60B
:1000B800ED930197E9F7ECE8F0E005901590BF01A2
:1000C800F001309751F0A591B591859195910590E2
:1000D8000D920197E1F7FB01F0CFEFE5EDBFE4E00A
:1000E800EEBFC0E6D1E00C947900609700E010E024
:1000F80020E030E040E050E0E8E0EBBBEABBEE2770
:10010800E2BBE0E4E1BBE0E1EA930E94EB020E947B
:1001180007032F5F3F4F829B04C000240416050687
:1001280009F00CC00E940703829B04C00024041637
:10013800050609F001C09698065F1F4F839B04C00F
:1001480000240416050609F00FC0E9E1F0E0FA936F
:10015800EA930E944F03839B04C0002404160506FB
:1001680009F002C041E050E0E1E0F0E0E417F507F3
:1001780041F4A22FB32FE5E0F0E00E947D03309711
:1001880009F002C0015010400E9407030E94AA0211
:10019800FE01FA93EA93E4E5F0E0FA93EA93E02F9C
:1001A800F12F0E9463030E94990384E00E944F028A
:1001B8002896FE01FA93EA930E94D102EE27EA9369
:1001C800E1E0EA930E949A02E3E6F0E0FA93EA9308
:1001D8000E94DB02E1E0F0E0E417F50721F40024D7
:1001E8000016010609F003C0969A40E050E08FCF50
:1001F8006096FFCF5F9BFECFECB108955D9BFECF6D
:10020800E881ECB921960895A881B9810E948B03F1
:10021800309751F00E948B033196ED93FC93319700
:10022800DF01EA81EC9304C0EA81EA930E940201AB
:100238002396089526970E949E0300E0E889F9898D
:100248003196E88BF98B3197E4913E2FE03011F429
:100258000C944B02E02FE03039F4353211F401E010
:1002680002C00E940D0312C1E130B1F4353221F40D
:100278000E940D0300E00AC102E050E010E03D32A8
:1002880011F411E003C13B3211F45BE2FFC03032DC
:1002980011F450E2FBC002C0E23039F440E003E060
:1002A800303311F41068F2C004C0E33011F00C943C
:1002B8004A02303310F03A3308F009C0A42FEAE0BC
:1002C800EA9FE02D4E2FE32FE0534E0FDFC0E32FC0
:1002D800E33631F40E941403EC910E941B03D5C04D
:1002E800E33741F40E9414030E9422030E943A0358
:1002F8000E2F0AC0E03761F40E9414030E94220303
:100308000E9444030E2F186012601F7720E038C047
:10031800E43611F0E93611F4146002C0E53731F41F
:10032800E4E7F0E0EE83FF8305E00DC0E83511F463
:10033800186004C0E83711F00C944902EEE7F0E0C9
:10034800EE83FF8304E012FF15C00E9414030E948D
:100358008B03EA87FB87AA85BB8510972CF40E943C
:100368005F03EA87FB875DE2503011F00F5F01C041
:100378001B7F06C00E9414030E948B03EA87FB8739
:1003880010FD11C0041778F417FF08C012FF04C04D
:100398001B7F352F015001C030E301C030E20E94BD
:1003A8000D034150EFCF202F11FF1AC02030B9F0B4
:1003B80013FF08C0EE81FF813196EE83FF833197EA
:1003C800E49105C0AE81BF81ED91AE83BF83EA930E
:1003D8000E942903403009F041502150E7CF4CC01A
:1003E80030E3EE81FF813296EE83FF8332970E94DD
:1003F8009503E887F987AA85BB85AE17BF0720F064
:100408003F5FAE1BBF0BC9F7AA87BB87E9E3E317BA
:1004180028F413FF02C0395F01C0395D14FD1EC006
:10042800E0E3E31730F0A885B985A130E0E0BE0726
:1004380011F410610AC0421710F010FF01C013C078
:1004480030E217FF0BC030E3106112FF07C01B7FBB
:100458005A930E942903403009F041500E940D032D
:10046800403009F041502150A885B985E1E0F0E01D
:10047800EA17FB0708F4B4CF10FF07C0403029F093
:100488004150E0E20E941B03F9CF00E0D7CE0E9462
:10049800A50362960895F82E2497DE010E945B0357
:1004A800AA83BB83DE0116960E945B030E948B031E
:1004B800E883F983DE0114960E945B030E948B0394
:1004C800FA93EA93EC81FD81FA93EA93FE0134965C
:1004D800FA93EA930E941E01A881B981EE27EC9352
:1004E80024960895AAB3AF70AABBD99AD8980CD00D
:1004F800DA9A0AD0CF99FBCFDA980895A07FAB2B70
:10050800ABBBDA9A01D0DA98FFE0FA95F1F70895D3
:10051800D998AAB3A76FAABBBBB3BF70A881EEDFF7
:10052800A881A295EBDFD99A219608950E947602B8
:10053800E881FF27E05AFE4FE081A981EA0FEA939C
:100548000E948C0249805880229608950E94760263
:10055800ECE00E942F03E1E0EA930E948C02EE2770
:100568005E2E4E2E0895EF93FF93A8816894AA30CB
:1005780021F0E8944394641438F45394EE27EA93F2
:100588005A920E949A022EF0ADDFD89AA881AA93B7
:10059800BFDFFF91EF9121960895F981E881A1913C
:1005A800AA2319F0AA93DFDFFACF22960895E881EB
:1005B800F981C895002021F031960A92D4DFF9CF4D
:1005C80022960895AA27BB271197F1F70895DA987C
:1005D800D8986880E881E058E0936201E881E054A7
:1005E800E09363013DD03CD03BD00E94E602E0E2BC
:1005F80032D0E8E230D0E6E0EA930E948C020E9412
:10060800AA0221960895E4E6F0E0FA93EA930C949E
:100618004F033A93ED85FE85FA93EA930C9408010B
:10062800AE85BF851497AE87BF8714960895EA9361
:10063800ED85FE85FA93EA930C9408010E948F03D6
:10064800EE83FF83FA93EA930895ED85FE85FA9386
:10065800EA930C940801EA930E948C020C947602A7
:100668000E94E602E0E3EA930C948C02A991B99106
:10067800EE27FF276D91662311F03196FBCF089581
:10068800AA27BB27E991F9910590002011F011964E
:10069800FBCFFD010895E991F991309639F080ED8D
:1006A80097E00197F1F7A8953197C9F708950024C5
:1006B800AF0DB01D0895E095F09531960895662721
:1006C8007727F7FF08956FEF7FEF0895002411242F
:1006D80090E1AA0FBB1F001C111C0E1A1F0A18F468
:1006E8000E0E1F1E01C0A1609A9599F7FD01D00159
:1006F8000895E894B7FF04C0A095B0951196689442
:10070800F7FDD9DFE3DFFD010EF4D5DF0895ED91A4
:10071800FC9111970895ED91FD916D917C9113973E
:1007280008950590F491E02D08957A936A93FA93C9
:10073800EA9308955A934A933A932A931A930A93F9
:1007480008955D814C813B812A8119810881089532
:00000001FF
